S1130000BD002ABD002FBD0044BD005ABD0061BD26
S1130010006ABD0077BD007DBD0081BD0085BD00C7
S113002097BD00A5CE002AAD003940488B0539475D
S11300302406CE002A472405CE002F200647240399
S1130040CE004439472407CE002A47240639CE007F
S11300502F20FA4724F7CE0044398605014A26FCAE
S11300603986064A27030120FA3986054A27044AB5
S113007026FA39BD0076396E0001386E002701CFAB
S11300803927013D39860536BD0090324A26F839B4
S1130090860A014A26FC39CE000501860A014A2651
S11300A0FC0926F6398605BD00B4860ABD00B4866F
S11000B0147E00B44A26FD390126013639BC
S9030000FC
